:0200000480007A
:100000006F00C004732F2034930F8000630AFF0336
:10001000930F90006306FF03930FB0006302FF038A
:10002000170F0080130F0FFE63040F0067000F000F
:10003000732F203463540F006F004000136E9E53E3
:10004000171F00002320CFFD6FF09FFF732540F1A5
:100050006310050073251030635805000F00F00F82
:10006000130E100073000000130E00009702000032
:10007000938282F973905230735020307350303035
:1000800073504030970200809382C2F7638C020065
:10009000739052109302B01A739022307323203061
:1000A000E39E62F873500030970200009382420191
:1000B00073901234732540F173002030B780000034
:1000C000938000E03771DBB6130171DBB38120024E
:1000D000B71E0000938E0E20130E00026394D14BC6
:1000E000B7800000938000FC3771DBB6130171DB31
:1000F000B3812002B71E0000938E0E24130E10024F
:100100006392D1499300000013010000B3812002E3
:10011000930E0000130E20006396D1479300100049
:1001200013011000B3812002930E1000130E300053
:10013000639AD1459300300013017000B38120020F
:10014000930E5001130E4000639ED14393000000B4
:100150003781FFFFB3812002930E0000130E500081
:100160006392D143B700008013010000B3812002E5
:10017000930E0000130E60006396D141B70000801B
:100180003781FFFFB3812002930E0000130E700031
:10019000639AD13FB7B0AAAA9380B0AA37010300EF
:1001A0001301D1E7B3812002B70E0100938EFEF751
:1001B000130EE0016398D13DB70003009380D0E7B0
:1001C00037B1AAAA1301B1AAB3812002B70E010068
:1001D000938EFEF7130EF0016396D13BB70000FF3C
:1001E000370100FFB3812002930E0000130E20029E
:1001F000639AD1399300F0FF1301F0FFB38120021D
:10020000930E1000130E3002639ED1379300F0FF5F
:1002100013011000B3812002930EF0FF130E400271
:100220006392D137930010001301F0FFB3812002D5
:10023000930EF0FF130E50026396D1359300D00059
:100240001301B000B3802002930EF008130E80005B
:10025000639AD0339300E0001301B0003381200291
:10026000930EA009130E9000631ED1319300D000AD
:10027000B3801002930E900A130EA0006394D03145
:10028000130200009300D0001301B000B3812002DC
:10029000138301001302120093022000E31452FEA4
:1002A000930EF008130EB000631ED32D130200004E
:1002B0009300E0001301B000B3812002130000009E
:1002C000138301001302120093022000E31252FE76
:1002D000930EA009130EC0006316D32B1302000067
:1002E0009300F0001301B000B3812002130000005E
:1002F0001300000013830100130212009302200078
:10030000E31052FE930E500A130ED000631CD32745
:10031000130200009300D0001301B000B38120024B
:100320001302120093022000E31652FE930EF0080F
:10033000130EE0006398D125130200009300E00043
:100340001301B00013000000B38120021302120059
:1003500093022000E31452FE930EA009130EF00046
:100360006392D123130200009300F0001301B00048
:100370001300000013000000B381200213021200DA
:1003800093022000E31252FE930E500A130E000156
:10039000639AD11F130200009300D00013000000E5
:1003A0001301B000B3812002130212009302200057
:1003B000E31452FE930EF008130E10016394D11D46
:1003C000130200009300E000130000001301B000CE
:1003D00013000000B38120021302120093022000D8
:1003E000E31252FE930EA009130E2001639CD11953
:1003F000130200009300F00013000000130000003F
:100400001301B000B38120021302120093022000F6
:10041000E31252FE930E500A130E30016394D1176B
:10042000130200001301B0009300D000B38120023A
:100430001302120093022000E31652FE930EF008FE
:10044000130E40016390D115130200001301B00098
:100450009300E00013000000B38120021302120099
:1004600093022000E31452FE930EA009130E5001D4
:10047000639AD111130200001301B0009300F00041
:100480001300000013000000B381200213021200C9
:1004900093022000E31252FE930E500A130E6001E5
:1004A0006392D10F130200001301B000130000008B
:1004B0009300D000B38120021302120093022000A7
:1004C000E31452FE930EF008130E7001639CD10BDF
:1004D000130200001301B000130000009300E000BD
:1004E00013000000B38120021302120093022000C7
:1004F000E31252FE930EA009130E80016394D109FA
:10050000130200001301B0001300000013000000EC
:100510009300F000B3812002130212009302200026
:10052000E31252FE930E500A130E9001639CD10504
:100530009300F00133011002930E0000130EA0018E
:100540006312D1059300000233810002930E000074
:10055000130EB0016318D103B3000002930E000024
:10056000130EC0016390D003930010021301200208
:1005700033802002930E0000130ED0016314D001CB
:10058000631CC0010F00F00F63000E00131E1E005D
:10059000136E1E00730000000F00F00F130E10000A
:1005A00073000000731000C0000000000000000095
:1005B000000000000000000000000000000000003B
:0405C0000000000037
:1010000000000000000000000000000000000000E0
:1010100000000000000000000000000000000000D0
:1010200000000000000000000000000000000000C0
:1010300000000000000000000000000000000000B0
:081040000000000000000000A8
:040000058000200057
:00000001FF
